:020000020000FC
:1000000062CE00000000000020C0BCC18EC0000015
:10001000000098C000000000000000000203040679
:10002000080C10182030406080000406080C1018DE
:100030002030406080A0C0000003070F1F000D0D9E
:100040000403060D0503030202004FB662FD0CC057
:10005000552041F00994C52DC095089483FDC7959E
:10006000C4BD64604FBE1895C0916400089483FDC0
:10007000C795C4BD6B7FC0916400CF3F09F41EC01B
:1000800070FF1AC082FD05C04FBEC1989798959821
:10009000189576FD0EC065FD0CC0C091B100C0FD85
:1000A0009298C1FD9398C2FD9498CAEFC095CA95E5
:1000B000F1F7C198979895984FBE189524BCCC2716
:1000C000C064C8BF6460F8CFC6CF70FFC4CF65FD01
:1000D000C2CFC19AC0CF70FFBECF65FDBCCF979A8B
:1000E000BACF70FFB8CF65FDB6CF959AB4CF929ACC
:1000F00070FFB1CF65FDAFCFC7E0CA95F1F7C19AE8
:10010000AACF939A70FFA7CF65FDA5CFC7E0CA9588
:10011000F1F7979AA0CF949A70FF9DCF65FD9BCF82
:10012000C7E0CA95F1F7959A96CF4FB6C9B7CF7E7B
:10013000C9BF6E7FCCB5CE0DDDB5DF1DDBBDCABD41
:100140004FBE18953FB68F7EA9B7A072A2118061ED
:10015000A9B7AF7DA9BFA9B7AE7FA9BF7894A09179
:100160006800AA2341F085FD2BC0A0916800AA95E4
:10017000A093680025C040E050E085FD15C0A6B3FF
:1001800096FDA095A0FD4FEFAEB5A06496FDAF7BA8
:10019000AEBDAA27A062A8BF8D7FA6B396FDA0958D
:1001A000A0FD5FEF451739F7A0E461FDA09368005B
:1001B00085FD03C0A0E4A093680040939600816091
:1001C00085FD0EC0A0916900AA2331F0A0916900BD
:1001D000AA95A093690004C08061AA27A062A8BF65
:1001E00080FF0AC0A09196004A2F61FF8E7F85FD97
:1001F00001C000C0409361004091B400443009F058
:1002000004C0A0916100A0936300A52DA03408F064
:100210006860A0916000A395A093600059F0F894E5
:10022000A9B7A160A9BF84FF03C0A9B7A062A9BFF5
:100230003FBE1895A0917400A395A093740042E06E
:1002400050916800552329F085FF03C05A955093BB
:100250006800A0919600A13018F0209299000DC07E
:1002600020929A002092A300A0919900AF5FA093E2
:10027000990018F0AFEFA0939900B09061005091F1
:10028000B400523049F466FF91F0A2E3BA1678F058
:10029000A0918600A0936100533049F466FF39F0C5
:1002A000A2E3BA1620F0A091C000A0936100509183
:1002B00062005B1521F010F05A9501C053955093E0
:1002C00062004A95D1F65091A300539509F45A95CE
:1002D0005093A300A091A400AA95A093A40009F0B4
:1002E00046C0A1E0A093A40045E0A091A5005A1744
:1002F000F0F1A091A6005A1728F441E0A3E0A093E2
:10030000A40007C0A091A7005A1718F441E0409339
:10031000A400D0909C00C0906300DC14A8F0A091D1
:10032000B400A430D9F066FD0FC0C0929C00539574
:1003300011F0A091A500A093A300A1E0A093A400B8
:10034000ACE3A093620013C0A0919C00A40F20F422
:100350005FEF50939C0002C0A0939C00A0919C0072
:10036000AF3F29F4AFEFA0939A00A093A300F894B5
:10037000A9B7A160A9BF84FF03C0A9B7A062A9BFA4
:100380003FBE18953FB646B557B58F7EA9B7A07248
:10039000A2118061A9B7AF7DA9BFA9B7AE7FA9BFE0
:1003A000789481FD25C0AEB5AF7B96FDA064AEBD4F
:1003B0008260A6B396FDA095A0FF05C0409365009E
:1003C000509366001FC1AEB5A06496FDAF7BAEBD75
:1003D000AA27A062A8BF8D7F85FF01C006C140E0AB
:1003E000A6B396FDA095A0FD00C140939600EFC076
:1003F000AEB5A06496FDAF7BAEBD8D7F61FF72C0D0
:10040000AEB5AF7B96FDA064AEBDAA27A062A8BF23
:1004100082604093910050939200A0908F004A19FF
:10042000B09090005B09BB24A22C4C38520518F404
:100430002092950049C0A091D400AA2359F1483CCC
:10044000520528F4A0E1BA2EAAE0AA2E23C048360D
:10045000A1E05A0728F4A8E0BA2EAFE0AA2E1AC0ED
:10046000403DA2E05A0728F4A4E0BA2EAEE1AA2E3D
:1004700011C0403AA5E05A0728F4A2E0BA2EACE336
:10048000AA2E08C04839A8E05A0720F4A1E0BA2EE5
:10049000A8E7AA2EC42EA0919300CA1AD52EA09127
:1004A0009400DA0ADD202AF4AFEFC094D094CA1A7F
:1004B000DA0A20929500A8E0A210A0E0CA14DA0699
:1004C00018F4A1E0A09395004093930050939400FA
:1004D000409191005091920040938F005093900072
:1004E00042E075C0A09165004A1BA09166005A0BBE
:1004F00094FD60C093FD5EC092FD5AC086FF03C0AC
:10050000D52EC42E0CC05695479591FD51C05695D9
:10051000479590FD4DC0D52EC42ED694C79461FD4D
:1005200019C0AC2DAC51AD2DA24008F005C0DD20A6
:1005300089F4AC2DA85C70F4A0916700A395AA2360
:1005400011F0A0936700AA3008F44FC020929600E3
:1005500081604BC0A0916700AA2319F0AA95A093CF
:100560006700A22C5091BA0097FD02C0A090C8006D
:10057000AAEFAA0EA22DA21DCA18DA0A4FB741701F
:10058000442319F040E050E015C0AFEFCA16D20482
:1005900018F04FEF50E00EC0A091AC00CA9E412D64
:1005A000000C441F50E008F012C04FEF50E00FC0A5
:1005B0005695479594FF07C0552309F04FEFA42F98
:1005C000A6954A0F521D4F3F520508F04FEF40933A
:1005D0009600816061FF09C0AFE1A095A923AB2916
:1005E0009A2F8F7DBB2009F48062A0E4A09368005D
:1005F00085FF03C0AAE0A093680061FD03C085FDEC
:1006000001C08F7E85FD03C0A0E2A0936900F8942D
:10061000A9B7A160A9BF84FF03C0A9B7A062A9BF01
:100620003FBE189511E00AC013E008C01AE006C0EA
:100630001EE104C014E602C018EC00C005E1BB27AF
:10064000BA95F1F70A95D9F71A95C1F708952AE3F3
:1006500038E709C020E33CE806C02AE234EB03C0D7
:1006600025E238EC00C012E0BB27939ABA95F1F767
:10067000979ABA95F1F79798BA95F1F79398BA9532
:10068000F1F7123009F0C19A123009F4959AB0913D
:10069000AD00BA95F1F7123009F0C198123009F4A3
:1006A0009598B7E8BA95F1F71A95F1F6022FB22F9F
:1006B000BA95F1F70A95D9F73A95A9F6939A08955C
:1006C000221B39E0001F3A9509F40895221F211BCF
:1006D00018F4210F8894F6CF0894F4CF622C722C72
:1006E000B0E08894B395221F331FE0F73795279524
:1006F0008894912E802E020B130B10F4192D082DC7
:1007000010F4889401C00894661C771CBA9571F7A0
:10071000172D062D0895322D11232AF43A950095B0
:100720001095031B130BF894029F712C002D129F40
:10073000912C802C7894780C172D921C292DB4E0E4
:100740006B2E2695179507956A94D9F7332321F0D8
:1007500000951095031B130B08950091B40004300D
:1007600009F474C0B0919600B95198F0B72FB670E3
:1007700081F466FD2BC005E09090C600B92DBA95B6
:1007800021F00AE0BA9509F002E1B0917B00B01BBC
:10079000E0F066FF0AC0B0919E00B0939C00BFEFEE
:1007A000B093A300B1E0B093A400B0916100B09306
:1007B000630020927E0020927F0020928000209291
:1007C0008100209282006F7B41C060649090C600DF
:1007D000B92DBA9579F4B0916200B095BB1FBB1FDB
:1007E0001B2FB7950B2FB12FB170B3951B2FB02FC7
:1007F000BE7F25C0B92DBA95BA9581F4B09162003B
:10080000B095BB1FBB1FBB1F1B2FB7950B2FB12F65
:10081000B370B3951B2FB02FBC7F14C0B091620092
:10082000B095BB1FBB1FBB1FBB1F1B2FB7950B2F4B
:10083000B12FB770B395B3951B2FB02FB87FB054BD
:100840000B2F120900937E0010937F0008951091E2
:100850007B00169500917A000795B0917E00B01B41
:100860000B2FB0917F00B10B1B2F28F40038BFEF86
:100870001B0740F009C00F37120508F405C00FE749
:1008800010E002C000E81FEF009383001093840083
:10089000089500918300B09180000B0F10918400A7
:1008A000B09181001B1F20E03091840033230AF4B3
:1008B0002A95B09182002B1F1AF4203F40F00AC005
:1008C0002F3008F407C00FEF1FEF2FE003C000E048
:1008D00010E020EF30916300B0919B003B1718F4BB
:1008E000323030F009C0B0918400BB235AF004C00C
:1008F000B0918400BB2332F40093800010938100F8
:100900002093820008952091D70000918300000F6A
:1009100010918400111FFFDE11232AF40038BFEF6D
:100920001B0740F009C00F37120508F405C00FE798
:1009300010E002C000E81FEF002352F0B091620007
:10094000B01B0B2F18F0013008F00AC001E008C0FE
:1009500000950F5FB09162000B0F08F001C00FEF20
:100960000093850008952091D80000918100109196
:100970008200D1DE11232AF40130BFEF1B0740F0C3
:1009800009C00F3F120508F405C00FEF10E002C0C8
:1009900001E01FEF112352F0B0918500B01B0B2F27
:1009A00018F0013008F00AC001E008C000950F5FA0
:1009B000B09185000B0F08F001C00FEF00936300AA
:1009C00008950FEF677F71FD29C072FD09C068604F
:1009D000B0917B00BA3020F0B52DB03408F4677FB9
:1009E000B091D300BB23D1F0B0917B00BB23B1F019
:1009F0000FEF10917B0064DEF894B091730072FDEC
:100A0000B5E00B9F112D002D7894112309F00FEF05
:100A1000B0919E000B1710F400919E0000939D0072
:100A2000089500917A0010917B0000541140B0911C
:100A30009D0010F4BA9501C0B39511F0B0939D00DC
:100A40000895E2D3B2E074FDB1E0B7B9B6B1B068D1
:100A5000B064B6B9E7DDB2E074FDB1E0B7B9B6B1E4
:100A6000B068B064B6B9B6B1B6FDFDCF04B115B18A
:100A7000B6B1BF77B6B91FD42CE62093A8002223C5
:100A800009F441C030E03093A900732E7694622EB1
:100A90006694620E731E262D372D0217130778F009
:100AA0008090A800BCE6B80DB093A8008090A90083
:100AB000B0E0B81DB093A900260D371DEECF809091
:100AC000A8009090A9001091A90016950091A80087
:100AD00007951695079523E0169507952A95E1F752
:100AE0002091B5002A9529F42092A8002092A9000F
:100AF0000AC02A9521F0800E911E2A95E1F7809276
:100B0000A8009092A90008952091B500B6B1B6FD55
:100B1000FBCF04B115B1B6B1BF77B6B9B091AA0099
:100B2000B395B093AA00B83060F12092AA00B091BA
:100B3000D200BB2321F1112329F0B091AB00BF3FBC
:100B400061F009C0B091AB000B1739F020F4BB2362
:100B500021F0BA9502C0B395E1F300919B00B093E8
:100B6000AB00BA3F50F400ECB93F38F400E8B83FAE
:100B700020F400E4B73F08F400E000939B007F7E80
:100B800008952130B1F00F3FB3E01B0790F4BCE6AD
:100B9000BB2379F0B091A8000B17B091A9001B07F7
:100BA00040F4B0919B00BB2359F0BA95B0939B00E1
:100BB00007C0B0919B00BF3F19F0B395B0939B0065
:100BC00000919B00B0916300B01B10F40091630092
:100BD000B0919C000B1750F000919C00B0919C00CC
:100BE000BF3F21F0B0919C00B0939B00502E00932A
:100BF0006400B091AA00B73009F47061089502E36F
:100C0000F894B091D9000B9F012D000C001F78942F
:100C1000B0919B000B1710F000919B0000936100B6
:100C200000936300502E0093640000939E0008958B
:100C300020927A00B0EFB0937B000895F8940CB541
:100C40001DB5209174007894309175006090760005
:100C50000093750010937600031B160971FD03C005
:100C600077FD7DC027C0709077002093770027091B
:100C7000222311F00FEF1FEF809078009090790001
:100C800030937800609279000091750010917600A1
:100C90000819190920917A0030917B003695279523
:100CA000020F131F10F40FEF1FEF00937A00109341
:100CB0007B0029C020917A0030917B003901B4E09B
:100CC0008B2EB2E09B2E343010F08A949A943830F8
:100CD00010F08A949A94769467948A94E1F726198E
:100CE0003709992021F0169507959A94E1F7200F7E
:100CF000311F20937A0030937B0028F43FEF30932C
:100D00007A0030937B00323008F4706871FF02C0C3
:100D1000B3E00DC0B091C40000917100023838F00A
:100D2000B395003A08F0B395B63008F0B5E09B2EC5
:100D3000B4E08B2E10917B0000917A0024E0169590
:100D400007952A95E1F70819120928F0B02FB2503B
:100D5000B12FB20910F402E010E0980126C02091F2
:100D60007A0030917B00390176946794669466949A
:100D700066942619320906950695200F321D209398
:100D80007A0030937B00323008F07F7704E03695AC
:100D900027953695279526952695201B10F022300D
:100DA00008F422E089019090C40060FDFECFE0903D
:100DB0008B00F0908C006160B9B7B061B9BF3801A9
:100DC00077FD41C07694679400938B0010938C005C
:100DD000B92DB330E1F0B0FD04C0060D171D93012D
:100DE00006C0000F111F0250120922E030E0B92D99
:100DF000B33068F020938D0030938E00009387000D
:100E0000109388006092890070928A003AC0009323
:100E10008D0010938E00209387003093880060929D
:100E2000890070928A0071FF0DC0BFE0B0938D0001
:100E300020928E00B093890020928A00B0938B009C
:100E400020928C001EC0669400938B00B92DB330A5
:100E500091F0B0FD03C0060D262D03C0000F025017
:100E600022E0B92DB33038F020938D000093870035
:100E70006092890006C000938D00209387006092E5
:100E8000890000917C0002FD0350013029F495FD9A
:100E90000AC0B0E0B7B909C0023019F4B7E0B7B979
:100EA00004C095FDF6CFB6E0B7B90091A200000FDF
:100EB00010F4BBE60B270093A20060FDFECFB2E06A
:100EC000B0936E006160B9B7B061B9BFB72FB670AB
:100ED000D1F020917A0030917B0036952795369598
:100EE000279571FF02C0B0E43B0FF8940CB51DB517
:100EF000020F131F1BBD0ABD6160B0E1B8BFB9B7D7
:100F0000B061B9BF78940895606120927D0020E0BF
:100F100067FD20E206C0606120927D0020E267FD4F
:100F200020E001E011E077FD11C0B72FB67009F0A5
:100F30006F7E14E100917B00069509F403950F3054
:100F400008F00FE071FF02C004E114E160FD0FC082
:100F5000B0917D00BB2359F071FF06C0B0916E00C7
:100F6000BA95B0936E0011F4706247C0ABDFB0B7B2
:100F7000B77FB0BFB8B1B0B7B860B0BFB0917D00B7
:100F8000B395B0937D00B8B177FD06C0B1E071FDB7
:100F9000B3E0BA95F1F7B8B1B072B21709F022C058
:100FA00071FF05C00395011708F00A95CFCF64FDC6
:100FB00005C00395011708F0B4CFC8CF6F7EF89431
:100FC0003CB56DB470907A0080907B00370D681C42
:100FD0006BBC3ABD6160B0E1B8BFB9B7B061B9BF31
:100FE00078949FCFB0916D00B13008F49ACF64FD32
:100FF00098CF0A9509F0AACF7F7D20918D0030917E
:101000008E00F894B0E1B8BF0CB51DB5020F131FE8
:101010001BBD0ABDE0908700F09088006160B9B701
:10102000B061B9BF7894B72FB67039F0B0916D0048
:1010300072FFB395B0936D0009C075FF07C067FDDF
:1010400005C064FD03C0BF91BF91E8C4089500E0EE
:1010500063FF03C064FF01C001E0F89410917100C8
:10106000B7E01B9F212D102D7894200F2695179502
:10107000269517952695179510937100183718F433
:10108000B8E7B093710000917100B09172000B1736
:1010900020F06062C1989798959860FDFECFE0902F
:1010A0008900F0908A006160B9B7B061B9BF089556
:1010B000B2E095FD0AC0F894B0937C00939A9298A0
:1010C00062FF01C0959A7894F4C0F894B0937C00C4
:1010D000939A949862FF01C0C19A7894EAC0B3E0F1
:1010E00082FF24C095FD11C002E0F894B0937C000B
:1010F000E1E8F0E00093B1009598949A62FF02C095
:10110000979A01C093987894D4C002E0F894B09371
:101110007C00E1E8F0E00093B100C198929A62FF90
:1011200002C0979A01C093987894C3C095FD0BC0F4
:10113000F894B0937C00EBE6F0E0959862FF01C074
:10114000979A7894B6C0F894B0937C00EBE6F0E000
:10115000C19862FF01C0979A7894ABC0B4E095FD46
:101160000AC0F894B0937C00929A949862FF01C0F0
:10117000979A78949EC0F894B0937C00949A929831
:1011800062FF01C0979A789494C0B5E082FF24C0B2
:1011900095FD11C001E0F894B0937C00E7E7F0E022
:1011A0000093B1009798939A62FF02C0C19A01C060
:1011B000929878947EC004E0F894B0937C00EBE8B9
:1011C000F0E00093B1009798939A62FF02C0959A5D
:1011D00001C0949878946DC095FD0BC0F894B093BD
:1011E0007C00E5E6F0E0979862FF01C0C19A789430
:1011F00060C0F894B0937C00E1E7F0E0979862FF5C
:1012000001C0959A789455C0B6E095FD0AC0F8944F
:10121000B0937C00949A939862FF01C0C19A78942D
:1012200048C0F894B0937C00929A939862FF01C0F2
:10123000959A78943EC0B1E082FF24C095FD11C01C
:1012400004E0F894B0937C00EBE8F0E00093B10088
:10125000C198929A62FF02C0959A01C094987894BE
:1012600028C001E0F894B0937C00E7E7F0E0009339
:10127000B1009598949A62FF02C0C19A01C09298F9
:10128000789417C095FD0BC0F894B0937C00E1E70B
:10129000F0E0C19862FF01C0959A78940AC0F89472
:1012A000B0937C00E5E6F0E0959862FF01C0C19A3A
:1012B00078946F7D089524E630E0F9012092B10022
:1012C000C19897989598929A939A949A6B7F08955B
:1012D000A2EBB0E007E00D9307E00D9301E00D9362
:1012E00004E00D930FEF0D930D9309E00D9302E0D1
:1012F0000D9301E00D9301E00D93AEEBB0E001E042
:101300000D9300E00D9304EB0D930FEF0D930D93F0
:101310000D9303E00D930FEF0D9301E00D930FEF8D
:101320000D9305E20D9300ED0D9308E70D9308EC86
:101330000D9304E00D930FEF0D9301E00D9300E08A
:101340000D930AE70D930AE00D9300E00D9301E081
:101350000D9300E00D930FEF0D9300E00D930895B2
:101360002091B9008B7F233009F48460B091BA00DA
:101370009F7DB1FD90629F7BB091BB00B1FD9064F9
:10138000223011F0886001C0877F08950A95E00F30
:10139000F21DB4910895ECE1F0E00091B200F6DFA7
:1013A000B093D700ECE1F0E00091B300EFDFB09331
:1013B000D800EAE2F0E00091B800E8DFB093D9008D
:1013C0000091D100002309F40395013108F001E1F7
:1013D000B02FB00FB00FB093A5001B2FB10FB10FFE
:1013E000B00FB093A600B10FB00FB00FB093A7002D
:1013F0000091B800023008F402E000937300B0914D
:10140000CE000FEFB23009F400EAB33009F402E87D
:1014100000937200E8E3F0E00091D500B7DFB093ED
:10142000A000089508952091C8003091C900B0919E
:10143000BA00B33009F43E5097FF02C020E03FEFFE
:10144000B32FB21B6B2EB25810F4B2E86B2E00E033
:101450000395609EB12DBD57D8F30093AC0008955D
:101460009068E1DFE5D820E030E0B0E16B2EDCD819
:10147000B09196002B0F321D6A94C9F7B4E03695EF
:101480002795BA95E1F7822E9F77CDDF0895F894DE
:10149000E3E0F0E0B9E0B7BFB491B078C1F3F894FD
:1014A000A895B1B5B861B1BDB0E0B1BDB4E0BEBF03
:1014B000BFE5BDBF00DFB0E0B8BBB2E1B7BBB0E095
:1014C000B5BBB0E0B4BBBCE1B2BBBCEBB1BB22244A
:1014D000A0E0B0E02D92AA31E9F7A0E6B0E00FEF6E
:1014E0002D920A95E9F7B1E0B093A200F1DED3D2D4
:1014F000B6B1B460B6B90091CA000093AD00B1E0D6
:10150000B0936A00F89498D8A2D892D8A3D890D86B
:10151000A4D88ED84FD390D88FD88CD8F8940AEF0F
:101520001AEFA6B396FDA095A0FF1FC01A95C9F7A4
:101530000A95B1F7E0E0FCE1B591B43E39F4B5911C
:10154000B03E21F4B591BF3F09F40CC0E0E0F39543
:10155000F395B591B83F49F4B591B43931F4B591EB
:10156000BA3A19F4EE27F6950994FADE14DF5ADF39
:101570005ADF0091CA000093AD009DDEB2E0B3BF18
:10158000B2E0BEBDB2E0B5BDB1E5B8BFB9BFB0B75E
:10159000B77FB0BFB8B1B0B7B860B0BF43D8789428
:1015A00050DA20927000BEB5B06496FDBF7BBEBD20
:1015B000B9B7B062B9BFBB27B062B8BF8D7F3CD8A6
:1015C000626033E02CE0B0919500BB2321F42CE065
:1015D0003A9509F4A3CF2CD880FFA0CF8E7FB0918D
:1015E0009600B23078F3B92FBF7100919800009344
:1015F0009700B0939800B01729F72A9521F76D7FCF
:10160000BEB5B06496FDBF7BBEBDBB27B062B8BFA0
:101610008D7FB091D400BB2321F48062B92FB070CC
:101620009B2F8F7B2092670005D885FF05C0B09166
:101630006700BA3008F08064F7D702E085FF01C088
:1016400000E0B0919600B017B8F3F89400D8FFD737
:10165000FED77894F1D720928600E6D7B091BE00ED
:10166000B13008F46EC0B0916A00B13008F469C0BE
:1016700085FD18C0B0919600BF3F08F462C0F89491
:10168000EFD77894D7D7B0919600B130C0F7F894DF
:10169000DED7CCD7DCD77894CDD7B0919600BF3FBA
:1016A000B0F3BAC2B8E09B2E9068F894BCDE789490
:1016B000C1D7F8949F77B7DE80909600B0919600DE
:1016C000BF37789408F445C0ADD7F894C9D778945B
:1016D0009A9451F7C5DEB82DB550B093C900ACD778
:1016E000F89406D26CD27894BAE09B2E9068F89465
:1016F0009ADE78949FD7F8949F7795DE8090960035
:10170000B0919600BF37789478F78CD7F8949FD72C
:101710008DD79DD778949A9449F7A2DEB82DBB5FF8
:10172000B093C80089D7F894E3D158D2789482D77F
:10173000F89479DE7894B0919600BF3F08F498CF82
:101740006BC200919600B09186000B1710F00093C9
:10175000860070D701E0B091BA00B35009F405E0FB
:10176000B0919600B01708F078CFF89479D778D771
:1017700077D7789461D720926A0020926B002092EC
:101780006C00B0916B00B395B0936B00BF3F71F5E7
:10179000B0916C00B395B0936C00B091CC0009E1AE
:1017A000BA9559F002E3BA9541F00DE7BA9529F0E0
:1017B0000AEFBA9511F020926C00B0916C00B0174E
:1017C000A8F079DD2FD7B0916C00BA95B0936C007A
:1017D00020926B00B091CB00B093AD00F89440D74D
:1017E0007894B091CA00B093AD0024D71FD7B091C0
:1017F0006800BB2319F485FF01C090CE01E085FD90
:1018000001C006E0B0919600B01708F4BACF12D725
:10181000B0916800BB2309F481CEF8944CDD20928E
:1018200061002092620020926300522C209264009A
:101830002092A1007894B091B700BB0FB0939F00A5
:1018400020927E0020927F002092800020928100D2
:10185000209282002092AA0060E070E02092710045
:10186000B8E0B093AA007061DDD6B2E074FDB1E0DB
:10187000B7B9B6B1B068B064B6B9B6B1B6FDFDCF10
:1018800004B115B1B6B1BF77B6B9112309F00FEFA6
:101890000093AB0039D9B8E0B093AA00706160DD65
:1018A000F894BFEFB0939B00AAD9B0916100B093B8
:1018B0009B00B0939C00B0939D007894B1E0B093EE
:1018C0006100B09363005B2EB0936400B093A400FA
:1018D000B0919A00B093A300B091BA00B33019F45C
:1018E0009F7D87FD90627160726020926D008CDC3C
:1018F000A2DC9ED9A3D99CD9A1D99AD90CDB2DD72A
:10190000A6DBD6DB9BD900DB66FDA1D777FF59D8D4
:1019100077FD87D89CDBE3DB91D9FDDA66FDB9D78B
:1019200096DB1CDC8BD9F0DA66FDEDD790DB2DDC85
:1019300085D9F1DA66FD17D88ADB66DC7FD9E4DA6F
:10194000B2E074FDB1E0B7B9B6B1B068B064B6B991
:101950007EDB71DC73D9D8D871FF1EC0B0919E00B8
:10196000B0939B00B0939C00B0919A00B093A300F9
:10197000B1E0B093A40018E12CE0B0916D00B11774
:1019800028F07D7F746020936F0006C0B0919600B0
:10199000B13008F0B3CF4CC072FF11C067FD0FC06B
:1019A000B0916F00BA9519F47B7F7860A7CFB093A0
:1019B0006F00B0919600B13008F0A0CF39C02092EE
:1019C0007000B0919900B13058F0B0919E00B09382
:1019D0009C00B0919A00B093A300B1E0B093A40032
:1019E000B09199000AEF1091D600112309F003E09D
:1019F000B01708F01DC085FF04C0B0916800BB237C
:101A0000B9F000EF67FF05C0B0919E00B0939B0056
:101A100000E2B0917B00B01708F470CFB091700075
:101A2000B395B0937000B0919600BB2309F002C04B
:101A300020927000F8943FDC8090B900B2E0B0933F
:101A4000B9008EDC8092B900209261002092620081
:101A500020926300522C2092640020929F0060E04C
:101A600070E07894E7D527DC0091D600002319F0C8
:101A7000C19A979A959AB6B1B460B6B985FF05C078
:101A8000B0916800BB2309F449CDB091BF00B130DB
:101A900008F0D2CD72CEEDE0F0E023D0053A09F0A7
:101AA0001BC0EEE0F0E01DD00A3509F015C03AE0A9
:101AB000A2EBB0E0E3E0F0E014D00D9331963A955C
:101AC000D9F739E1AEEBB0E0EFE0F0E00AD00D93EA
:101AD00031963A95D9F702C0FBDB0AD0E8E2F0E094
:101AE0000895E199FECFEEBBFFBBE09A0DB30895D8
:101AF0001ED03AE0A2EBB0E0E3E0F0E00D910FD0B1
:101B000031963A95D9F739E1AEEBB0E0EFE0F0E08D
:101B10000D9105D031963A95D9F712D00895E199F3
:101B2000FECF0DBBEEBBFFBBE29AE19A0895EDE05C
:101B3000F0E00FEFF4DFEEE0F0E00FEFF0DF0895FC
:101B4000EDE0F0E005EAEBDFEEE0F0E00AE5E7DFEC
:101B500008953091AE000091AF00313011F4009340
:101B6000B200323011F40093B300333011F400931B
:101B7000B400343011F40093C600353011F40093F2
:101B8000B500363011F40093B800373011F40093EB
:101B9000C400383011F40093B900393011F40093C7
:101BA000CE003A3011F40093BA003B3011F40093A8
:101BB000BB00089525E040D52A95E9F7089547D55B
:101BC00049D54BD54DD532D542D544D546D548D546
:101BD0002DD53DD53FD541D543D5089541D53DD5EA
:101BE00039D535D523D53CD538D534D530D51ED5C6
:101BF00037D533D52FD52BD508958090AE00909052
:101C0000AF0025D524D523D511D58A94D1F728D571
:101C10000DD59A94E1F70895F894D1DF7894CADF4E
:101C2000C9DFB1E0B093AE00B1E0B093AF00209255
:101C3000B000F894E2DF7894B5E06B2E70909600D7
:101C4000FBD4B09196007B16C9F7B13018F0BF3FB6
:101C500040F107C07EDFF8944BDFB1DFB8E0B1BDE3
:101C6000A9DF6A9459F7B091B000B395B093B00072
:101C7000B33008F4DECF9EDFB091AF00B395B093E0
:101C8000AF00F894B091AE00BA95EEE3F0E0EB0F40
:101C9000F21D049178940395B091AF00B01708F449
:101CA000C6CF88DF87DFB091AE00B395B093AE00AA
:101CB000B091AE00BC3008F4B7CF0ADBF89418DF5F
:081CC000B8E0B1BD77DFE3CB12
:00000001FF
